:020000020000FC
:10000000C5C009C01895189508C118951895189578
:10001000189518951895889480990894441F331F53
:10002000221F111F90FD05C08A9500E080131895CE
:100030008AE11370512F622F40FF04C00BE160274B
:1000400003E0502741FF04C00FE8602703E050277A
:1000500042FF04C007EA602702E0502744FF04C0C3
:100060000EEE602701E0502745FF04C00CED60272D
:1000700003E0502746FF04C001E0602702E050275C
:1000800047FF04C00BEB602701E0502730FF04C09E
:1000900006E7602703E0502731FF04C005E560272D
:1000A00003E0502732FF04C003E1602703E050273C
:1000B00033FF04C00FE9602703E0502734FF04C07A
:1000C00007E8602702E0502736FF04C00EE66027ED
:1000D00001E0502737FF04C00CED602702E05027F5
:1000E00007EF43FD602707EB35FD60277330C1F153
:1000F0007230D1F0713061F0683DF1F55330E1F5C7
:100100003ED020937000309371009E7F73951895B8
:10011000643D91F5533081F532D0209372003093D5
:1001200073009E7F739518950091720003FD0CC0BB
:100130006C3511F5523001F522D0209374003093C4
:1001400075009E7F739518956C3CB1F45330A1F403
:1001500016D020937400309375009E7F7395189588
:10016000683551F4523041F40AD020937600309330
:1001700077009E7F92601895772791601895179564
:1001800027953795179527953795089500E101BD77
:100190000FE60DBF00E808B90FEF07BB00EE01BB8B
:1001A00005E00FEF02BB00E003BF0FBD0CE00EBD8A
:1001B0000CEE0DBD08E30CBD03E10BBD08EC0ABD60
:1001C00000E409BF03E005BF00E40BBFF89400E3BF
:1001D00008BBC09AC098A0E7BB27BA95F1F7AA95CB
:1001E000E1F700E208BBC09AC09808E008BBC09ADB
:1001F000C0980CE0F9D001E0F7D006E0F5D002E8B5
:10020000F3D0F4E0E0E414D1FF240FECE02E1ED094
:100210008AE1789491FD22C0FDCFF8940E2DE4D0B0
:10022000C0E1AAE7B0E0AF0D0D91CFD0CA95CC23C5
:10023000D9F700ECE01611F0EA9401C0F39400E461
:10024000F01619F4FF240FECE02E1895AAE7B0E0A1
:1002500000E2CFE40D93CA95E9F70895F89406E01B
:10026000C3D09D7F772700917000C09178000C1754
:1002700039F400917100C09179000C1709F40BC09A
:100280000091700000937800009171000093790054
:1002900001E0AAD0DBDF7CD000917200087F11F072
:1002A0000830D9F40091730088940370001F00682F
:1002B0009BD00091760089D00091770086D0009184
:1002C000730004FD05C00FE88FD00DE27ED05EC044
:1002D0000FE88AD00AE279D059C000917200007FFD
:1002E0000032C1F400917300009173000F70000F91
:1002F000000FC02FAAE7B0E0AC0F009174000D937F
:10030000009175000D93009176000D930091770098
:100310000D933CC000917200007F0034B9F5E0916C
:100320007500E1708894C0917700F0917600CC1F41
:10033000FF1FEE1FCC1FFF1FEE1FFF1FEE1FFF1F33
:10034000EE1F09E851D0C795C795C5FD04C0C795F4
:10035000CF71EC0F03C0C795CF71EC1B0E2F08D0E7
:10036000F795F7950AE331D0FF730F2F01D00EC038
:10037000B02FAA27BA5010F0A395FCCFB65F0A2F72
:10038000006323D00B2F006320D00895789442CFD0
:100390008499089509E828D000E217D000917800E8
:1003A00002950BD00091780008D000917900029559
:1003B00004D00091790001D008950F700A3010F434
:1003C000005D01C0095C01D0089518D0D0EFD023A2
:1003D000D8BBC29A05D0DFE0D023D295D8BBC29A51
:1003E000C09A1FD0C098089509D0D0EFD023D8BBB1
:1003F000F7DF0295D0EFD023D8BBF2CFDFE0D7BB39
:10040000DD27D8BBC19AC09A0CD0D6B3C09809D00A
:10041000C09A07D0C098D7FDF1CFC198DFEFD7BB06
:100420000895000000000000000000000000089592
:10043000C895002021F0002DC8DF3196F9CF08952E
:0C044000524453204465636F64657200F1
:00000001FF
